:030000000219FDE5
:03000B000200AA46
:03002B0002018748
:03005B0002033667
:0300730002032362
:1000800002030406080C10182030406080040608A3
:100090000C10182030406080A0C00003070F1F0D17
:1000A0000D0403060D0503030202C2AF306308C24C
:1000B0006385798AD2AF32C0D0C0E0206221E525C5
:1000C0006016E473E525F4C3334009758A00D263F2
:1000D000F57901D6F58AD262D0E0D0D0D2AF32C362
:1000E000E526334009758A00D263F57901F0F58A77
:1000F000C262E526F4602F30682520720DD0E0D072
:10010000D0C295C293C297D2AF32C295C293C29762
:10011000206F0C2066097412D5E0FDE57B4290D07B
:10012000E0D0D0D2AF32758A00D263757900C28D2B
:10013000D262211F01C4306805206602D29501C435
:10014000306805206602D29701C430680520660237
:10015000D29301C4C29430680A2066077412D5E0B5
:10016000FDD29501C4C29630680A2066077412D584
:10017000E0FDD29701C4C29230680A20660774126B
:10018000D5E0FDD29301C4C2AFC2AD53E6EFC0D0FB
:10019000C0E0D2D3D2AFE57A6009E5776005757724
:1001A00000412C757701C2CEE52A600720744915FD
:1001B0002A21F87800790020742EE580307E01F441
:1001C00030E50278FF53DACF207E0343DA20307E19
:1001D0000343DA10C2D8C271E580307E01F430E505
:1001E0000279FFC3E89970CB306103752A4020740F
:1001F00003752A40885CD27020740DE52B600415CD
:100200002B410843DA01C2D8207002411BA85C20B0
:100210006102C270207402411988227882B60403F8
:10022000852224C3E52594404002D26420CF0AD021
:10023000E0D0D043E610D2AD32C2CF053AE57A60C5
:1002400009E578600575780061197578017802E52F
:100250002A6005307402152AC3E55C9401400575D7
:100260005F004175756000756900E55F2401F55F09
:100270005003755FFF7982B7020D306E1DC3E52212
:1002800094324016854C227982B7030E306E0BC330
:10029000E52294324004798E8722C3E523952260BB
:1002A000084004152341A90523D8CA0569E56970EA
:1002B000021569D56A63756A017805C3E569956BAE
:1002C0004057C3E569956C50087801756A030202CE
:1002D000DDC3E569956D50057801756A01C3E56276
:1002E0009524401E7982B70402610E206E14852485
:1002F00062E569046003856B69756A0175233C02D8
:100300000319E5622850057562FF610EF562E5622A
:100310000470067560FF7569FFD0E0D0D043E61029
:10032000D2AD32C2AF53E67F7592FA7593FFC260C9
:10033000759104D2AF32C2AF53E6EFC2ADC0D0C0A8
:10034000E0C0F0D2D3D2AFA8FBA9FCE57A6007C326
:10035000E913F9E813F8C2D830710261A853DACF73
:10036000207E0343DA10307E0343DA20D271E58029
:10037000307E01F420E502617F88278928A18D5312
:10038000DACF207E0343DA20307E0343DA10C2D86E
:10039000C271307402A1797800E580307E01F430BA
:1003A000E502A179885CA16153DACF207E0343DAAC
:1003B00020307E0343DA10C271206102818153DA5A
:1003C000CF207E0343DA10307E0343DA20C2D8D236
:1003D0007188578958C3E89555F8E99556F97B0017
:1003E0007E087A00C3E8948CE994005005755B00A0
:1003F0008173882178A2E6A8216055C3E894C8E9F2
:1004000094005008E4D2E4FB7A0A814EC3E8946871
:10041000E994015008E4D2E3FB7A0F814EC3E894DB
:10042000D0E994025008E4D2E2FB7A1E814EC3E880
:1004300094A0E994055008E4D2E1FB7A3C814EC3D4
:10044000E89498E994085008E4D2E0FB7A787E00BA
:10045000C3E89559FCE9955AFD30E70AECF424010C
:10046000FCEDF43400FD755B00C3EC9AED9E500387
:0F047000755B018859895A85575585585678020A
:10047F00A161C3E89527F8E99528F9307C02A145D9
:10048F00307B02A145307A02A13E20750281A4E99A
:10049F00FDE8FC81C3E9C313F9E813F8307902A131
:1004AF003EE9C313F9E813F8307802A13EE9C3130C
:1004BF00FDE813FC20612CC3EC941CED9402400268
:1004CF0081DAED701EC3EC94C850180529E5297028
:1004DF00021529C3E529940A5002A179755C00D24F
:1004EF0070A179E529600215297400207F037896A1
:1004FF00E624FAFEE43400FFC3EC9EFCED9FFD50B2
:10050F000678007900A145C3EC94FFED94004006F6
:10051F0078FF7900A145EC8572F0A4C5F0A2F733FE
:10052F00F87900400302056178FF7900020561E95F
:10053F00C313F9E813F8307C0EE9600278FFC3E8C3
:10054F001338F8E43400F9C3E894FFE9940040024B
:10055F0078FF885CD270206102A179741FF4552F47
:10056F004BF52FC274EB7002D274752A40307403AE
:10057F00752A0A306102A18D20740353DAFE2074AC
:10058F0003752B20D0F0D0E0D0D0D2AD43E610329F
:10059F0079010205BD79030205BD790A0205BD790E
:1005AF001E0205BD79640205BD79C80205BD781725
:1005BF00E4D5E0FDD8FAD9F6227A147B780205E467
:1005CF007A107B8C0205E47A0D7BB40205E47A0B7A
:1005DF007BC80205E47902E4C296D5E0FDD297D537
:1005EF00E0FDC297D5E0FDD296D5E0FDE920E0020F
:1005FF00D29530E002D293E573D5E0FDE920E00219
:10060F00C29530E002C2937496D5E0FDD9C9EAF8DD
:10061F00D5E0FDD8FBDBBEC29622C37C007D007502
:10062F00F00005F0EA33FAEB33FB50F6EB13FBEA7D
:10063F0013FAC3E9FFE8FEE89AF8E99BF95004EFD3
:10064F00F9EEF8B3EC33FCED33FDD5F0DFEDF9EC5B
:10065F00F822E889F08A20D2D4F8A9F07B0030F78D
:10066F000B7BFFF42401F8E9F43400F9E88520F05E
:10067F00A4ADF0F8E98520F0A4AFF0FEED2EF974EB
:10068F00003FFA7C04C3EA13FAE913F9E813F8DC24
:10069F00F48BF030F70AE8F42401F8E9F43400F9A8
:1006AF00E889F0C2D4F8A9F0227882B604030207D1
:1006BF0057C3E55C9419401EE52D54067018206E43
:1006CF003678057994E7146007780A146002781277
:1006DF00C3E54198401F306E098564627569FF75E7
:1006EF006A01852224E4F544F545F546F547F548BA
:1006FF00C26E020757D26E7994E7147013E523F494
:10070F003333F913F8E9540104F9E854FE02074BA7
:10071F00E714147014E523F4333333F913F8E95461
:10072F000304F9E854FC020753E523F4333333335E
:10073F00F913F8E954070404F9E854F8C39440F89E
:10074F00E99400F98844894522C3E54113F9E5404E
:10075F0013F8C3E54498F8E54599F9500CC3E894AC
:10076F0080E994FF401602078FC3E8947FE9940055
:10077F00500302078F787F790002078F788079FF07
:10078F008849894A22E5492546F8E54A3547F985DA
:10079F004A20E4300701F43548FA30E709C3EA94F8
:1007AF00F040150207CDC3EA940F50030207CD782E
:1007BF00FF79FF7A0F0207CD780079007AF0C3E551
:1007CF00249561500AC374019524500B0207EBE581
:1007DF004A20E70E0207EBE54A30E70688468947CD
:1007EF008A482278A5E6FAC3E54933F8E54A33F992
:1007FF00120661E930E70BC3E89480E994FF4013D8
:10080F000126C3E8947FE9940050020126787F798E
:10081F00000126788079FFE820E715C3E52398F8D3
:10082F004009C3E89401400302084D780102084DC6
:10083F00E8F424012523F8400302084D78FF884B84
:10084F002278A6E6FAA847A948120661E930E70C14
:10085F00C3E89401E994FF4016020882C3E894FFAD
:0F086F00E99400500302088278FF7900020882A2
:10087E00780179FFE920E715C3E54B98F84009C3E5
:10088E00E8940140030208A978010208A9E8F424BB
:10089E0001254BF840030208A978FF88242278FF2F
:1008AE00C26420693D206A12D264C3E541940A40B5
:1008BE0009C3E52594405002C26479A1E76023E59F
:1008CE0041601F74FF8541F0848539F0306A0375ED
:1008DE00F005A4F8C5F0600278FFC3E895645002F5
:1008EE00A864886322C3E54094C8E5419400E5639B
:1008FE005003142104046002F563227883E6F52088
:10090E00120FA375E89012059F75E890E5E820ECAC
:10091E00FBA8BDA9BE121049756E55756F00C37444
:10092E000013FD7455606613FC74552CFC74003D69
:10093E00FDECFAEDFBC3E89AE99B4014E56E2455F5
:10094E00F56EE56F3400F56FEA2CFAEB3DFB80E5B2
:10095E00AE6EAF6FC3E56F13F9E56E13F8C3E9130F
:10096E00F9E813F87A03C3E913F9E813F8DAF7AAEA
:10097E00201A7009756E00756F0002099B1AEA60E5
:10098E0008EE28FEEF39FFDAF88E6E8F6F2275E8CB
:10099E0090227883E6FFE5E820ECF7A8BDA9BE0516
:1009AE0070C3E57094084052757000E9FA79A0E7BB
:1009BE006044EA7007E571601B0209D6C3E89571C1
:1009CE006010E5715006600C140209E20460F90231
:1009DE0009E2E571F571C39472401B7561C0C39451
:1009EE00044013756180C39404400B756140C39439
:1009FE0004400375610075BB0822EFC39401601FAC
:100A0E007455601BC3E894FFE994035012C3E89534
:100A1E006EE9956F5009E561600C1561020A34E5C7
:100A2E0061F460020561A861C3E524985002A82410
:100A3E00C3E89562400AA862E562F46003856261CC
:100A4E0088258826E570B4070375BB1022743279A9
:100A5E00A787F0A4C5F0A2F733F8C3E8956140026A
:100A6E00A8618822882488258826886422754000FB
:100A7E007541F022C2AF75C820A8CCA9CDAA3A30D4
:100A8E00CF010A75C824D2AFC3EA13FAE913F9E805
:100A9E0013F8AB3BAC3C883B893CC3E89BF8E99C24
:100AAE0020690A547FF9306702619C41F9AD3D8A95
:100ABE003DF9EA9D547FFA600478FF79FFAE3EAFB0
:100ACE003F8B3E8C3FA83BA93CC3E89EF8E99FF9BB
:100ADE00C3E54113FBE54013FAE82AF540E93BF57F
:100AEE004150067540FF7541FF6143AA40AB41ACD2
:100AFE0040AD417E047F02C3EB940440021E1FC32F
:100B0E00EB940840021E1FC3ED13FDEC13FCDEF741
:100B1E00C3EA9CFAEB9DFBEF6009C3E913F9E813F6
:100B2E00F8DFF7EA28FAEB39FB8A408B4150067B57
:100B3E00FF8B408B41C3EB94025002D267306904A5
:100B4E007F03616E7892E6FFC3E537948240110F02
:100B5E00C3E53794A040010FC3EF940640027F0512
:100B6E007E02E541C4540FF9E541C454F0F8E54066
:100B7E00C4540F28F8C3E89EFAE99400FB4009C359
:100B8E00EA9402EB940050047A02E4FB61E8AA4076
:100B9E00AB41EBC4FEEAC4540F4EFCC3EA9CFAEB25
:100BAE009400FBC3E813C313F8EA28FAEB3400FBF6
:100BBE008A408B41C3EB94024002C2677802EBC4B9
:100BCE00FE7B00EAC4540F4EFAC3EA98FA4005C3FE
:100BDE00940250027A027892E6FF30600261E88554
:100BEE005192855293D26043E680C3E49AF8E49B17
:100BFE00F9C3E833F8E933F9306702817BE8FAE9A3
:100C0E00FBD3E913FDE813FC88518952C3EF94031B
:100C1E006038EF20E00DE82CF8E93DF9ECFAEDFB39
:100C2E00020C44E828F8E939F9C3E82402F8E9345B
:100C3E0000F97AFE7BFFC3EF9403400E8A538B5468
:100C4E00884D894E8C4F8D5081AF885389548A4D73
:100C5E008B4E8C4F8D503069127553F07554FF7555
:0F0C6E004FF07550FF7551F07552FF81AFE8FAE6
:100C7D00D3E813FC8851C3EF94036020EF20E00705
:100C8D00E82CF8ECFA819BE8282402F87AFEC3EFF1
:100C9D00940340088A53884D8C4F81AF88538A4DF9
:100CAD008C4FE568C3335002646BF5683060028188
:100CBD00B9753402D26043E680E52D5406602DA847
:100CCD0040A941C3E913F9E813F8306904E9244058
:100CDD00F9C2AF53E67F759100C3E498F594E4999A
:100CED00F595759104D26043E680D2AF22D2657539
:100CFD004300752000306C03752040020D19D2653C
:100D0D00754300752040306C037520007801790122
:100D1D00206720E52D54066002C2657914E541C3B4
:100D2D0013700104F8C394144002781430690478E8
:100D3D001B791BC3E833F8C3E933F9206010E54391
:100D4D00600C306903D53404D26DA1D091C1054337
:100D5D00E59B5440B52002A1BA30690908C3E89952
:100D6D00400118A14820650A08C3E8994002A1195D
:100D7D00A148C265C2AF53E67F7591003067127509
:100D8D0094007595FC759104D26043E680D2AFA1B5
:100D9D0019AE40AF41C3EE33FEEF33FF50047EFF7B
:100DAD007FFFC3E49EF594E49FF595A192C3E533CF
:100DBD0094015002A119306502A119D802A1CEA14A
:100DCD0048C26DC2AF53E67F75910085539485542B
:100DDD0095759104854D92854E93D26043E680D2F0
:100DED00AFE52D54066008206A020533020E0C3063
:100DFD006D0D206C0A2065071581158102168C2258
:100E0D0078003064053065027801E53775F007A488
:100E1D00F9E5F028F5F0E9A2F013A2F113A2F2130F
:100E2D00F537C394785003753778C3E53795384057
:100E3D0008D266C295C293C297306002C146854FF3
:100E4D0092855093D26043E68022207D16C2AF7505
:100E5D004202C296D294306202D293D2AF759F11E4
:100E6D00021046C2AF754202C296D292306202D2D1
:100E7D0095D2AF759F11021046307243207D20C26E
:100E8D00AF754203900165757B40C293C29230628B
:100E9D0004D297C1A4D296D2AF759F13021046C249
:100EAD00AF754203900165757B40C295C294306267
:100EBD0004D297C1C4D296D2AF759F1002104620AE
:100ECD007D17C2AF754203900140C293306202D2CA
:100EDD0097D2AF759F13021046C2AF7542039001B2
:100EED0040C295306202D297D2AF759F1002104664
:100EFD00207D16C2AF754204C294D292306202D2E6
:100F0D0097D2AF759F10021046C2AF754204C292C0
:100F1D00D294306202D297D2AF759F130210463031
:100F2D007243207D20C2AF754205900154757B1030
:100F3D00C297C296306204D295E14AD294D2AF756F
:100F4D009F11021046C2AF754205900176757B0464
:100F5D00C297C296306204D293E16AD292D2AF7533
:100F6D009F11021046207D17C2AF754205900136C4
:100F7D00C297306202D295D2AF759F11021046C250
:100F8D00AF75420590014AC2973062EBD293D2AF52
:100F9D00759F11021046207D16C2AF754206C29292
:100FAD00D296306202D295D2AF759F13021046C20F
:100FBD00AF754206C294D296306202D293D2AF750B
:100FCD009F10021046307243207D20C2AF75420142
:100FDD00900176757B04C295C294306204D293E180
:100FED00F0D292D2AF759F10021046C2AF7542017A
:100FFD00900154757B10C293C292306204D2950158
:10100D0010D294D2AF759F13021046207D17C2AF38
:10101D0075420190014AC295306202D293D2AF75EA
:10102D009F10021046C2AF754201900136C2933037
:10103D006202D295D2AF759F13C2662290013475AC
:10104D007B00C295C293C297C294C292C296C262ED
:10105D0022788076070876070876010876040876E8
:0E106D00FF0876FF08760A087602087601086A
:10107B007601788C76010876000876B40876FF083E
:10108B0076FF0876FF0876030876FF087601087668
:10109B00FF0876250876D00876780876C808760497
:1010AB000876FF08760108760008767A08760A0833
:1010BB0076010876010876000876FF08760022781C
:1010CB0087E6FFC272BF0302D2727888C27DE63018
:1010DB00E102D27DC27E7889E630E102D27EC3EF97
:1010EB0094026008758E01D2730210FC758E00C2DB
:1010FB0073227880E6149000809378A5F67881E6C9
:10110B00149000809378A6F67886E61490008D9361
:10111B0078A7F6789FE6F8700108C3E894114002AF
:10112B007811E82828F56B256B256B28F56C256B5A
:10113B002828F56D7886E6F539C394025003753986
:10114B0002789CE67538FFB402037538A0B403032C
:10115B0075388278A3E61490009A93F566114922AC
:10116B00227896E6FA7897E6FB7888E6B40305C30F
:10117B00EB940EFB307F047A007BFFC3EB9AFCC32E
:10118B00948250027C827572000572EC8572F0A419
:10119B00C3E5F0947D40F222D27F316C1205AE7A1A
:1011AB00007B007C101205A4E55C2AFA74003BFB63
:1011BB00DCF37C04C3EB13FBEA13FADCF7FEC27F10
:1011CB00316C22E5EF20E6037520000520903FFFF0
:1011DB00E520146006901FFF1460009304600375F4
:1011EB00EF1253D9BF7581C043FF8012059F75EF76
:1011FB000243B203E5B3240220E70DF521E5E3201A
:10120B00E0068521B343E30111497580FF75A40006
:10121B0075F1B275D4DF75900175A5FC75F2FE758D
:10122B00D50175A60175E2411149E4F8F6D8FD75B3
:10123B006801115E1216EA78988673753001C2AF99
:10124B001205B81205C81205AE1205CF1205AE1263
:10125B0005D61205AE12180C1205B81205B81205F8
:10126B00B3C2AF78FA79FA308507D9FBD8F7021CED
:10127B000011CA11FD316B316C7898867311497569
:10128B00A90075B680757A0075881075890275C8C6
:10129B002475910475D84075A82275B80275E6902F
:1012AB00759B80759D0075D10E75BCC075BB08759F
:1012BB00BA1175E88012059FD2AF12090975360075
:1012CB0053DACF207E0343DA20307E0343DA104318
:1012DB00DA01C2D8C2711205B8D2617B037A0CE570
:1012EB005B70077A0CDB0302126C1205AE207003E5
:1012FB0002126CC270E55CC3940240E1E52F541FEF
:10130B00855E5DF55EB55DD5DAD5C26153DACF206A
:10131B007E0343DA20307E0343DA10C2D8C27178E1
:10132B00A2E67008D274E52F54E0F52FC27575292B
:10133B00001205B3307409C3E529940A4002D27533
:10134B001205A478023074027800C3E55C9840F073
:10135B00C2AF1205C81205C81205C8D2AF1205B824
:10136B00754C001205A4788CE6C39401500302144B
:10137B0044E530C394015003021444207435C3E593
:10138B005C94FF5003021444C2AF1205DDD2AF12BE
:10139B0005B3C3E55C940150EFC2AF1205C812054B
:1013AB00A91205C8D2AF1205B3C3E55C94FF40E99F
:1013BB000218917F05D27F316C1205B3C2AFC27F89
:1013CB00316CAE5CC3E55C947FD2AF407612059F67
:1013DB00C2AF1205DDD2AFDFDC31A3C3EE940578CB
:1013EB0097F61205B812172B1218147F0AD27F31F9
:1013FB006C1205B3C2AFC27F316CAE5CC3E55C94BB
:10140B007FD2AF50E612059FC2AF1205C81205A9D5
:10141B001205C8D2AFDFD631A3EE24037896F612AD
:10142B0005B812172B1218431205B3316CC3E55CC8
:10143B0094FF50026186021891C3E55C954C400302
:10144B00855C4C1205B378017988E7B40302780503
:10145B00C3E55C984002616EC2AF1205DD1205DD7B
:0E146B001205DDD2AF1205B8753000E4F53180
:10147900F5320531E531F4703E0532789AE678198E
:10148900146012783214600D787D14600878FA14AB
:101499006003753200C3E53298401C114912059F5B
:1014A900153275310078998673C2AF1205DDD2AF56
:1014B900789886731205B31205A9E52A7005307468
:1014C90002416C78012074027806C3E55C9840A259
:1014D9001205B3E52A700302126CC2AF1149E4F593
:1014E90022F523F524F525F526F567D2AF7885E6AB
:1014F900C333F565E4F544F545F546F547F548F593
:1015090070F52CF52DF53775700875BB1012059F10
:1015190012099CE5E820ECFBA8BDA9BEE97001F819
:1015290088711209A075700875BB1011CAC2AF7510
:1015390061FF120A5B852261852262852263D2AF2F
:101549007522017524017525017526018560697566
:101559006A0175B69075A903757A017888E6B403AE
:1015690007C27D307602D27DD268D2697533001206
:101579000FA3120FD2120A7B120A82120A7B120AD5
:1015890082120A7B120D0B1206B8120E0D120E579B
:10159900120A82120CFA306E0312075820670312DE
:1015A90008AC3067031208F3120E0D120E86120AE8
:1015B90082120D0B306E03120794120E0D120EFDDE
:1015C900120A82120CFA306E031207F2120E0D1271
:1015D9000F2C120A82120D0B306E03120850120ED4
:1015E9000D120FA3120A8212099C120CFA120E0D87
:1015F900120FD21209A0120A8230692C8564618502
:101609006462856069756A0179187A0CC3E5339952
:101619004009C269D26A8A35021631C3E55C940170
:10162900400302158D021694306A1D206C1AE535A7
:10163900147006C26AD26BA18DF535C3E55C9401BD
:10164900400302158D021694753600C3E55F9401B7
:101659004009856462856069756A0178FA79A4E749
:1016690060027803C3E55F985021307404E52A606D
:101679001A78F0306C058564617820C3E54198508B
:1016890002A18D0536E55C6002C197753600C2AFCF
:1016990011497887E6FE760211CA7887EEF6E4F5F5
:1016A90022F523F524F525F526F565752C00752D0C
:1016B9000075A90075B680757A00D2AF1205B3110D
:1016C9004978A4E66006D295D297D293307406E59C
:1016D9002A7002416C788DE6C394014002614B8106
:1016E90076901A0D782012176DE520B4A50CA31277
:1016F900176DE520B45A0302170B115E12172B025E
:10170900172A901A0378807B0A12176DA308DBF950
:10171900901A0F788C7B1912176DA308DBF9901AB0
:101729002822C2AF1217AC121786901A00740E1233
:101739001772A37406121772A37415121772901AEE
:101749000378807B0A121771A308DBF9901A0F78C6
:101759008C7B19121771A308DBF91217BF12179D99
:10176900901A2822E493F622E6438F01538FFD75E0
:10177900EF0275B7A575B7F1F0538FFE22438F02BB
:10178900438F0175EF0275B7A575B7F1901A0DF082
:10179900538FFC22901A0D74A5F172901A0E745A87
:1017A900F172227A3079D07820901A40F16DE520D3
:1017B900F709A3DAF7227A3079D0901A40E7F17263
:1017C90009A3DAF922AB74A875BB01027980BB02BF
:1017D900027981BB03027982BB04027994BB0502B9
:1017E9007983BB06027986BB07027992BB08027925
:1017F90087BB0902799CBB0A027988BB0B027989EC
:10180900E8F7227C051205B8DCFB22C2AF1205C835
:101819001205CF1205D61205DD1205A91205C81247
:1018290005CF1205D61205DD1205A91205C8120544
:10183900CF1205D61205DDD2AF22C2AF1205DD12D5
:1018490005D61205CF1205C81205A91205DD120524
:10185900D61205CF1205C81205A91205DD1205D643
:0F1869001205CF1205C8D2AF22AE74AF75C2AF51
:101878001205C81205C81205C81205A9DEF212051C
:10188800DD1205A9DFF8D2AF221114110C110C7565
:10189800740175750175760011727C05AD5C1205D1
:1018A800B8C3ED955C70F5C3E55C9401400AC3E5E7
:1018B8005C94FF40340218CF1217CE12172B111464
:1018C800C2AF75EF12110CDCD30576C3E57694032D
:1018D800500280C4110C0575E5741490009F93F8AC
:1018E80008C3E57598500280AC110C110C0574C33F
:1018F800E574940C5002809A12105E12172BC2AF36
:0519080075EF12110C47
:0319FD000211CE06
:101A00000E061507070104FFFF0A020101A55A018E
:101A100000B4FFFFFF03FF01FF25D078C804FF01DA
:091A200000FF0A010100FF00FFB4
:101A4000234656544C6962656532304150726F23AB
:101A500023424C48454C492346333930232020202B
:101A60002020202020202020202020202020202076
:101C0000C2AFC2D353D9BF7581C043B20343FF8073
:101C1000752438752503B1C975EF0275E24043F1AB
:101C20002053A4DF75D4FFD2857DFA780379E67C52
:101C300010752200752300901DD67B0675249875BB
:101C400025013085028142208508D8FBD9F9DCF7CF
:101C500081B4308508D8FBD9F9DCF781B4B189E4C7
:101C600093A3C39A6004DDC381B4DBDBB17B600264
:101C7000812B7B08E493FAA3B15CDBF87A30B15C8A
:101C8000752200752300B17BEAFCEBFDC3ED94FEE9
:101C9000400EB17B8A278B28ED30E0048A828B834B
:101CA000B17B7AC270D8C3ED94FE601350CEBD00F4
:101CB00025EC60097520007521FF0200008100A855
:101CC00027A9280809D804D90281D3B17FEA89AAB3
:101CD000F281C50D81A0C3ED94035049EDA2E092BD
:101CE000007AC5C3E5829400E583941C50902000DF
:101CF00010438F02438F0175B7A575B7F1F030001F
:101D00001FA827A9280809438F01538FFDD804D99C
:101D100002A12089AAE275B7A575B7F1F0A3A10DBC
:101D2000538FFC817C7AC1BD030CE493A3FAB140CC
:101D3000DCF8B138817C817EAA22AB23B15CEBFA5E
:101D4000EA6222752608C3E52313F523E52213F57D
:101D50002250066323A0632201D526EAB1C9B1C986
:101D600075260AEAF4200102D285300102C285B14B
:101D7000C9C3134002C201D526EB22B17FEAFB2082
:101D80008502A17F308502A184752608AE24AF2587
:101D9000C3EF13FFEE13FEB1CDB1C9C3EA13308513
:101DA000024480FA30E703632201C3E52313F523DD
:101DB000E52213F52250066323A0632201D526D91C
:101DC000E52265236523F52222AE24AF250E0FDE22
:101DD000FEDFFCD20122424C48656C693437316326
:041DE000F390060175
:00000001FF
